:1000000004309F009E009C01003065008501FF3098
:1000100066007F30620006080F399D000330061F1E
:100020009D061D080339031903309D040C30861FFB
:100030009D061D080C3903190C309D041D18051070
:100040001D1C05149D1885109D1C85140430061E6A
:1000500005301D1D09309D1D00309F001F081E0228
:10006000031C9E0A1E081F02031C9E0310308506F7
:100070009C099C1C05159C18851542309B00053079
:100080009A0001309900013098009B0B45289A0B8B
:100090004528990B4528980B45289C1C5F2824303F
:1000A0009B0003309A0001309900013098009B0BAF
:1000B00057289A0B5728990B5728980B5728861AB8
:1000C0006E28000010309B0002309A009B0B6628BF
:1000D0009A0B66286B286C286D286E2805118511EF
:1000E0001E08861E0A3E820788289628A428B12862
:1000F000BE28CC28DD28EB28F92807291529232933
:1001000031293E294B2958296A297729842992299E
:1001100012309B0004309A009B0B8C289A0B8C2881
:10012000912892289328942800000B2887309B0060
:1001300004309A009B0B9A289A0B9A289F28A02893
:10014000A128A22800000B280D309B0005309A0042
:100150009B0BA8289A0BA828AD28AE28AF28B0285A
:100160000B28A7309B0005309A009B0BB5289A0BF3
:10017000B528BA28BB28BC28BD280B2856309B00C0
:1001800006309A009B0BC2289A0BC228C728C828A1
:10019000C928CA28CB280B289C309B0006309A001F
:1001A00001309900013098009B0BD4289A0BD42879
:1001B000990BD428980BD4280B287A309B00073051
:1001C0009A009B0BE1289A0BE128E628E728E8280B
:1001D000E92800000B284B309B0008309A009B0B4D
:1001E000EF289A0BEF28F428F528F628F7280000C6
:1001F0000B2836309B0009309A009B0BFD289A0B88
:10020000FD28022903290429052906290B283F3046
:100210009B000A309A009B0B0B299A0B0B29102983
:1002200011291229132914290B28D0309B000430DE
:100230009A009B0B19299A0B19291E291F2920297D
:10024000212922290B283E309B0005309A009B0B68
:1002500027299A0B27292C292D292E292F293029A6
:100260000B28E0309B0005309A009B0B35299A0B38
:1002700035293A293B293C293D290B2898309B00F8
:1002800006309A009B0B42299A0B4229472948299C
:1002900049294A290B286B309B0007309A009B0B99
:1002A0004F299A0B4F2954295529562957290B288C
:1002B000BE309B0007309A00013099000130980051
:1002C0009B0B60299A0B6029990B6029980B602978
:1002D00000000B28C9309B0008309A009B0B6E2948
:1002E0009A0B6E2973297429752976290B28C43035
:1002F0009B0009309A009B0B7B299A0B7B29802954
:100300008129822983290B28DE309B000A309A003C
:100310009B0B88299A0B88298D298E298F29902952
:1003200091290B2819309B000C309A009B0B9629C1
:100330009A0B96299B299C299D299E299F290B2848
:02400E00F13F80
:1042000041006C0063006F007200200031002E003E
:1042100032002D004C0058003300200043006F0096
:104220007000790072006900670068007400200067
:10423000310039003900390020004D002E002000E7
:1042400043006F00760069006E00670074006F0025
:024250006E00FE
:00000001FF
